:0A00060000308A00132A00000A10DF
:100010008A100A118207543445344D345034453423
:100020005234413454345534523441343D342534FF
:1000300033342E343134663420344734523441342E
:1000400044344F3453340D340A345234453450342C
:100050004F345234543445343D34253434346434CC
:100060000D340A3400342A08B3002B08B400B5015B
:10007000A71F3C283317B403A71726080319DF2846
:100080007F302602031C9B28A600B6010430B7006F
:100090000310A90DA80DA70DB50DB70B4828043006
:1000A000260203185B2803302602031DD5280A30D8
:1000B0003502031CD5280330A602B60AA921031075
:1000C000A90DA80DA70DB50D92210230B7000310A0
:1000D000B50CA70CA80CA90CB70B6728A9210430F4
:1000E000B7000310AA0CAB0CAC0CAD0CB70B71280D
:1000F0009221A9212C08AD002B08AC002A08AB00E6
:10010000AA019221A9212B08AD002A08AC00AA015E
:10011000AB019221B5194F28A608031D9428A90AFE
:10012000A80AA70AB50AD5280310A90DA80DA70D7E
:10013000B50DA6034F28A609A60A7F30A607B6016B
:100140000430B7000310A90DA80DA70DB50DB70B0E
:10015000A2280430A60705302602031CE128A921A5
:100160000310A90DA80DA70DB50D0310A90DA80D1D
:10017000A70DB50D92210310A90DA80DA70DB50D62
:10018000B60A0330B7000310B50CA70CA80CA90CD5
:10019000B70BC3280330A602351EAB280310B50CDD
:1001A000A70CA80CA90CA603AB28A609A60A033025
:1001B000A607360AB402031CB4010130E22802305B
:1001C000E2280030AF00B31BF028B41BF028B408BD
:1001D0000319F02820300C1EEB289900B40BEA28F4
:1001E000331FF6282D300C1EF3289900B31F032966
:1001F000B41B0329B4080319032930300C1EFE2850
:100200009900B40BFA28B31333132F1C0E293608A8
:10021000AF003608B100330AB1073829AF1C1229E4
:10022000330AB600B308031990292E300C1E162984
:1002300099003608B200B20333083202031C2229A7
:100240003308B200B20803192B2930300C1E2629BE
:100250009900B20B25293608B700330AB7020318F4
:10026000B229A603330AB1003608B1023108AF0043
:100270003508AE00260803194229B0000310AE0C61
:10028000B00B3E2931080319902930302E070C1E7F
:10029000472999002F08031D5429B30803199029F1
:1002A0002E300C1E51299900AF03B1030319902978
:1002B000260803196029B0000310AE0DB00B5C29AD
:1002C0002E08B5023508AA002708AB002808AC00A4
:1002D0002908AD000310A90DA80DA70DB50D031039
:1002E000A90DA80DA70DB50D2D08A907031C7D2983
:1002F000A80F7D29A70F7D29B50A2C08A807031C84
:100300008429A70F8429B50A2B08A7070318B50A63
:100310002A08B5070310A90DA80DA70DB50D38299A
:100320000000B2292D08A907031C9B29A80F9B29AF
:10033000A70F9B29B50A2C08A807031CA229A70F01
:10034000A229B50A2B08A7070318B50A2A08B5077A
:1003500000343508AA002708AB002808AC0029089B
:10036000AD00003400008A114A2A2A08F801290247
:100370000318BD292908F700C929F7010830AB0087
:10038000A90DF70D2A0877020318F700F80DAB0B3B
:10039000C02900342708F700A71BD229281DDE2911
:1003A0002030D729F709F70A7708A7002D30F80081
:1003B00078080C1ED9299900281DA8152708A9001E
:1003C0006430AA00B5217708A70078083030031DF3
:1003D000F0292818F729A819F729281A2030F22916
:1003E000A8112812F80778080C1EF429990027088C
:1003F000A9000A30AA00B5217708A7007808303094
:10040000031D062AA8190B2A281A2030F807780895
:100410000C1E082A99003030A70727080C1E0E2A48
:1004200099008A115D2A84011F30830583161F08F5
:10043000C0399F009B01073083129F00193083163B
:100440009900223098009030831298003330A30036
:10045000A2003B30A1008330A0000C30A400A50115
:1004600025080720A50AF70077080C1E352A9900F1
:100470000C302502031D302A2308A9002208A800F9
:100480002108A7002008A600AD01AC010130AB0097
:10049000AA0033281130A60026080720A60AF70074
:1004A00077080C1E512A990022302602031D4C2A7F
:1004B0002408A7001030A800CA290D300C1E5E2A9F
:0E04C00099000A300C1E622A9900652A63001A
:040000008A01032846
:00000001FF
